:040000003FEF00F0DE
:100008005F82FACF01F0FBCF02F0E9CF03F0EACF2D
:1000180004F0E1CF05F0E2CF06F0D9CF07F0DACF50
:1000280008F0F3CF09F0F4CF0AF0F6CF0BF0F7CFD2
:100038000CF0F8CF0DF0F5CF0EF00EC0F5FF0DC0A7
:10004800F8FF0CC0F7FF0BC0F6FF0AC0F4FF09C0A9
:10005800F3FF08C0DAFF07C0D9FF06C0E2FF05C0FA
:10006800E1FF04C0EAFF03C0E9FF02C0FBFF01C0D3
:10007800FAFF5F921100D5EF0DF020501F101E10EF
:1000880004E1690E1D5CD8A002D0000E12001DC04C
:1000980024F01EC025F0090ED89024362536E82E07
:1000A800FBD7000E266E200E276E000E286E2450F9
:1000B8002624326E25502720336E000E2820346EF9
:1000C800000E386E000E376ED5D0000E2D6E000E65
:1000D800366E000E356E040E365CD8B026D037501A
:1000E8002124D96E38502220DA6E37503224256EFA
:1000F80038503320266E000E3420276E25C0F6FFB8
:1001080026C0F7FF27C0F8FFDE500900F518D8B45D
:1001180007D0010E2D6E3550375E3650385A05D04F
:10012800374A382A354A362AD6D72D04D8A4A2D039
:1001380037503224246E38503320256E000E342078
:10014800266E000E2414276EFC0E2514286EFF0E52
:100158002614296E27502E6E28502F6E2950306E87
:10016800316A000E0F6E080E106E2EC011F02FC0EF
:1001780012F030C013F0040E156E000E146E75ECFC
:100188000DF02EC011F02FC012F030C013F018EC93
:100198000FF037503224246E38503320256E000E6D
:1001A8003420266EFF0E2414276E030E2514286EA5
:1001B800000E2614296E27502E6E28502F6E2950B7
:1001C800306E316A000E2E240F6E080E2F20106E2E
:1001D80021C011F022C012F011501210D8A4200E24
:1001E800136E020E156E000E146E75EC0DF0100EE7
:1001F8002C6E000E2A6E080E2B6E37503224246E99
:1002080038503320256E000E3420266E000E24143C
:10021800F66EFC0E2514F76EFF0E2614F86E26D027
:10022800000E366E000E356E365014E1400E355C09
:10023800D8B010D02AC0D9FF2BC0DAFFDF50F56E36
:100248002A4A2B2A0D00374A382A354A362A365088
:1002580001E1ECD70A00840EA66EB50EA1EC0EF0F3
:10026800010EF626000EF722000EF8222C062C2886
:10027800D8A4D6D7020E385CD8A027D7010E120012
:10028800E7D071C09CF072C09BF073C09AF074C044
:1002980099F076C0B3F077C0B2F00001B251286E81
:1002A8000001B351296E2A6A2B6A090ED8902836A4
:1002B80029362A362B36E82EF9D728C019F029C056
:1002C8001AF02AC01BF02BC01CF019EC08F000092A
:1002D800D8A4D0D0010E0001C66F0001B2510001B0
:1002E800B311D8B4B1D00001B207D8A0B307020E39
:1002F8000001C66F0001B4510001B511D8B407D090
:10030800B4C0D9FFB5C0DAFF0001DFBEB3D0EFC07B
:100318001BF0F0C01CF099C01DF09AC01EF09BC0E5
:100328001FF09CC020F0000E216E060E226E01D830
:100338000AD00500FA6E0001E951FD6EEA51FE6E21
:10034800FF6AFA501200E806D8B41BD0640E000108
:10035800C76103D00001C72B8DD0020E04017C6F4A
:1003680000018151F00B0309816F000E00018B6FB2
:10037800000E00018C6F010E0F6E010E15EC07F0D8
:1003880063D0010E00019927000E9A239B239C231A
:10039800000E0401786F020E796F000E7A6F000E5E
:1003A8007B6F000E0001C06F060E0001C16F030EC7
:1003B8000001C66F040178510401791104017A1112
:1003C80004017B11D8A402D0010E3FD0040E000115
:1003D800C66F0001B4510001B511D8B407D0B4C03C
:1003E800D9FFB5C0DAFF0001DFBE44D0010E0F6EA1
:1003F800C0C010F0C1C011F0400E126E010E98EC92
:1004080007F00FC0B4F010C0B5F0030E0001C66FBE
:10041800400E0001685F000E695B6A5B6B5B400E13
:100428000401785F000E795B7A5B7B5B400E00010C
:10043800C027000EC1231ED0020E04017C6F010EDE
:100448000F6E010E15EC07F0000E0001C66F12D0FA
:100458000001C651000AD8B414D7010AD8B43DD750
:10046800030AD8B447D7010AD8B4A4D7070AD8B41E
:10047800B0D7E2D70001C65112000001D051D8A46C
:1004880015D0000E656E000E0F01366F160E0F01A7
:10049800396F9F0E0F01376F7B0E0F01366F01D03A
:1004A800658665A6FDD7010E0001D06F0001D00555
:1004B800D8B465BA0CD0000E626E000E0F01366F0C
:1004C8000F0136810F013689020E0001D06F62A438
:1004D80006D00F0136A503D062946CEC0EF065A22D
:1004E80002D0A198120062A009D00F0136A106D04F
:1004F8000EEC03F0040E0001D06F629062A804D0E5
:100508000F0136B988EC0EF062AC1FD00F0136AD82
:100518000ED0000E1F6E730E1E6E000E206E000EA3
:10052800216E000E236E010E226EDBEC0CF0629C35
:10053800E5EC0EF00001D351D8B402D00001D30786
:100548000001D351D8B4DDEC09F062AA04D00F0140
:1005580036BB2BEC0EF062A212D00F0136A30FD0DF
:100568007F0E1F6E1E68000E206E000E216E000E9C
:10057800236E010E226EDBEC0CF0000E636E040E8F
:100588000001D06102D0A19812000F0136A740D017
:10059800000E2E6E030E2E6401D03AD062A638D01B
:1005A80064CFE0F00001E031E832E8320F0B0001DF
:1005B800D66F62960001E0B508D00001D651010D52
:1005C800BA0EF324D96E000E07D00001D651010DE2
:1005D800B80EF324D96E000EF420DA6E0001DF7035
:1005E8000001D6510001D8A403D006EC0BF00ED0C0
:1005F800000E1F6E720E1E6EE00E206E000E216E33
:10060800000E236E000E226EDBEC0CF02E2AC2D7F1
:10061800A1981200A098000E636E000E626E000E84
:100628000F01266F270E0F6E0F0E106E000E126E42
:10063800000E116E000E146E010E136EBAEC0EF061
:10064800160E0F01396F9F0E0F01376F7B0E0F01CA
:10065800366F000E176E070E176401D00ED01750B4
:10066800040D000EF324D96E040EF420DA6EDE6A4F
:10067800DE6ADE6ADD6A172AEED7658C000E0F0186
:10068800386F6598659C6296000E546E000E0001E6
:10069800946F000E0001966F000E956F62B6F3D747
:1006A800010E0001D16F010E0001D26F000E000192
:1006B800CD6F000E0001CE6F000E0001CC6F000E52
:1006C800176E010E176401D02ED01750020D570E69
:1006D800F324D96E000EF420DA6E000EDE6E000EE2
:1006E800DD6E1750020DA90EF324D96E000EF4200A
:1006F800DA6E000EDE6E000EDD6E1750010DB80EBC
:10070800F324D96E000EF420DA6E000EDF6E175057
:10071800010DBA0EF324D96E000EF420DA6E000E25
:10072800DF6E172ACED7080E576E040E586E160EB7
:100738000F01266F040E0401036F200E026F080ECE
:100748000401016F040E0401006F0401008F000E04
:100758000001DE6F000E00019D6F000E9E6F000EFF
:100768009F6F000EA06F000E0001D46F000E0001F5
:10077800D06F1200800E04012019D8A41200C00EF8
:10078800546E82D0D70E516EF20E526E000E566E17
:10079800120E556E120004012251D8A441D0040152
:1007A8002251020D090EF324F66EF20EF420F76EB4
:1007B800F86A000EF8220900F5CF51F00A00F5CFCB
:1007C80052F0020E51240F6E000E5220106E0FC010
:1007D800F6FF10C0F7FFF86A0E0EF76403D00800A2
:1007E800F55005D0F6CFE1FFF7CFE2FFE750556EA1
:1007F800030E51240F6E000E5220106E0FC0F6FF2C
:1008080010C0F7FFF86A0E0EF76403D00800F55021
:1008180005D0F6CFE1FFF7CFE2FFE750566E1200A2
:10082800000E546E1200040E0401226127D0040148
:100838002251020D010EF324F66EF20EF420F76E2B
:10084800F86A000EF8220900F5CF51F00A00F5CF3A
:1008580052F051C0F6FF52C0F7FFF86A0E0EF76467
:1008680003D00800F55005D0F6CFE1FFF7CFE2FF3F
:10087800E7500F6E0F50556E566A1200000E546EF8
:100888001200000E546E120004012351010AD8B45C
:1008980079D7030AD8B47FD7010AD8B4C4D7F1D717
:1008A800176E0001B4510001B511D8B407D0B4C017
:1008B800D9FFB5C0DAFF0001DFBE12000001B65152
:1008C8000001B711D8B407D0B6C0D9FFB7C0DAFF56
:1008D8000001DFBE1200C9C018F00001C469000E93
:1008E8000001C66F000E0001C86F68C078F469C0C7
:1008F80079F46AC07AF46BC07BF4010E04017C6F52
:10090800030E0001C96F49D0020E04017C6F12006A
:10091800010E0F6E010E15EC07F01200020E040115
:100928007C6F010E0F6E010E15EC07F01200000E21
:100938000F6E010E15EC07F01200020E04017C6F19
:10094800000E0F6E010E15EC07F0120098EC0CF07B
:1009580000018151F00B0509816F200E00018B6F9A
:10096800000E00018C6F020E1818D8A410D00001D8
:1009780068510001691100016A1100016B11D8B4B6
:1009880006D0000E0F6E010E15EC07F01200010ED6
:100998000F6E010E15EC07F012001750010AD8B4BB
:1009A800B3D7030AD8B4B4D7010AD8B4B7D7070A5B
:1009B800D8B4BDD7010AD8B4C0D77A0AD8A41200CF
:1009C800C5D7EFC00FF0F0C010F001D80AD005006D
:1009D800FA6E0001E751FD6EE851FE6EFF6AFA50AB
:1009E80012000009D8B40CD000016D51010DCB0ED6
:1009F800F324D96E000EF420DA6EDE04D8A41AD0DF
:100A08006DC04CF0010E4D6E000E4E6E4C2A03D098
:100A1800D8904D364E364C2EFBD74D1C4F6E4E1C83
:100A2800506E4F500001BC1750500001BD1710EC1C
:100A38000DF054D06DC04CF0010E4D6E000E4E6E90
:100A48004C2A03D0D8904D364E364C2EFBD7000199
:100A5800BC514D160001BD514E164D504E10D8A434
:100A68003BD0EFC00FF0F0C010F001D80AD005005D
:100A7800FA6E0001E151FD6EE251FE6EFF6AFA5016
:100A880012000F501010D8B424D06DC04CF0010ED5
:100A98004D6E000E4E6E4C2A03D0D8904D364E3611
:100AA8004C2EFBD74D500001BC134E500001BD1316
:100AB80000018151F00B0609816F280E00018B6F30
:100AC800000E00018C6F010E04017C6F77EC79F049
:100AD80005D010EC0DF002D077EC79F00001C4518C
:100AE8001200000E0F6E300E106E040E116E400EC6
:100AF800126E010E98EC07F00FC0B6F010C0B7F0F8
:100B080059C0B4F05AC0B5F0000E0001C96F000119
:100B1800C469000E0001C66F000E0001C86F000E08
:100B28000001C56F000E0001A56F000EA66F000E34
:100B3800A76F000EA86F000E0001A16F000EA26F34
:100B4800000EA36F000EA46F010E0001C36F000E0C
:100B58000001BD6F000EBC6F000E00016D6F49D023
:100B680000016D51010DCB0EF324D96E000EF42057
:100B7800DA6E000EDF6EEFC00FF0F0C010F001D893
:100B88000AD00500FA6E0001E751FD6EE851FE6ECD
:100B9800FF6AFA5012000009D8B427D0EFC00FF04E
:100BA800F0C010F001D80AD00500FA6E0001E1513A
:100BB800FD6EE251FE6EFF6AFA5012000F501010DF
:100BC800D8B413D06DC01AF0010E1B6E000E1C6E47
:100BD8001A2A03D0D8901B361C361A2EFBD71B5066
:100BE8000001BC131C500001BD1398EC0CF000016F
:100BF8006D2B00016D51D8A41200B2D720EE01F080
:100C08005B50D9265C50DA22DF50106E105000017C
:100C1800955D000E9659D8A095C010F010500001AF
:100C2800955F000E965B000E0F6E12D00F50010DEF
:100C3800280EF324D96E040EF420DA6E91C0E1FF79
:100C480092C0E2FFDFCFE7FF0001914B922B0F2A02
:100C580010500F5CD8A0EAD70001955100019611F9
:100C6800D8B432D020EE01F05D50D9265E50DA2299
:100C7800080EDF6E20EE02F05D50D9265E50DA22B3
:100C8800280EDE6E040EDD6E5BC0D9FF5CC0DAFF95
:100C9800DFBC0DD05DC0D9FF5EC0DAFF480EDF6E45
:100CA8005DC0D9FF5EC0DAFF000EDB8E12005DC0AA
:100CB800D9FF5EC0DAFF080EDF6E5DC0D9FF5EC0E7
:100CC800DAFF000EDB8E120020EE01F05D50D9260F
:100CD8005E50DA22080EDF6E20EE02F05D50D92653
:100CE8005E50DA22200EDE6E040EDD6E5DC0D9FF86
:100CF8005EC0DAFF040EDF6E5DC0D9FF5EC0DAFFAA
:100D0800000EDB8E0001949F0001CF51D8A4120081
:100D1800DDEC09F01200659854BE3DD0000194AF97
:100D28000FD0020E0001D56F0001CE51D8B4FFECF0
:100D38000BF0000E0001D26F000E0001D16F1200FF
:100D480020EE01F05D50D9265E50DA22080EDF6EE3
:100D580020EE02F05D50D9265E50DA22200EDE6EBB
:100D6800040EDD6E5DC0D9FF5EC0DAFF0C0EDF6ECB
:100D78005DC0D9FF5EC0DAFF000EDB8E57C0D9FF19
:100D880058C0DAFF040EDF6E57C0D9FF58C0DAFF2B
:100D9800000EDB8E1200040120AF15D0010E0001F9
:100DA800D56F0001CD51D8B4FFEC0BF0000E000157
:100DB800D26F000E0001D16F0001CF51D8A41200EC
:100DC800DDEC09F01200020E0001D56F20EE01F0F3
:100DD8005D50D9265E50DA22080EDF6E20EE02F052
:100DE8005D50D9265E50DA22200EDE6E040EDD6ECE
:100DF8005DC0D9FF5EC0DAFF040EDF6E5DC0D9FFAB
:100E08005EC0DAFF000EDB8E000E0001D26F000E0E
:100E18000001D16F0001CF51D8A41200DDEC09F018
:100E28001200146E1450D8A42BD020EE01F05D509F
:100E3800D9265E50DA22080EDF6E20EE02F05D50F1
:100E4800D9265E50DA22200EDE6E040EDD6E5DC0FD
:100E5800D9FF5EC0DAFF0C0EDF6E5DC0D9FF5EC041
:100E6800DAFF000EDB8E57C0D9FF58C0DAFF040E38
:100E7800DF6E57C0D9FF58C0DAFF000EDB8E1200B4
:100E88000F50106E116AD890103611361450126E29
:100E9800136AD89012361336D8901236133610507B
:100EA800122611501322D89012361336D8901236C3
:100EB8001336000E1224156E040E1320166E15C07C
:100EC800D9FF16C0DAFF000EDB8415C0D9FF16C0A3
:100ED800DAFF000EDB8E1450040DF3CF10F0F4CFC0
:100EE80011F00F50020DF3501026F4501122D89033
:100EF80010361136D89010361136040E1026000E12
:100F08001122000E1024156E040E1120166E15C045
:100F1800D9FF16C0DAFF000EDB8415C0D9FF16C052
:100F2800DAFF000EDB8E1200176E0F50D8B407D010
:100F38001750020D570EF324D96E000E06D0175025
:100F4800020DA90EF324D96E000EF420DA6EDECF5E
:100F580018F0DDCF19F018501910D8A405D0000EDC
:100F68000F6E000E106E120020EE02F01850D926F7
:100F78001950DA2210C0DEFF11C0DDFF20EE01F0AB
:100F88001850D9261950DA2212C0DFFF18C0D9FF2D
:100F980019C0DAFF400EDF1618C0D9FF19C0DAFFF2
:100FA800000EDB8618C0D9FF19C0DAFF000EDB8EF1
:100FB8000F50D8B418D01750020D570EF324D96E1D
:100FC800000EF420DA6EDECF13F0DDCF14F0040E3D
:100FD8001318156E1450166E1750020D570EF32481
:100FE800D96E000E17D01750020DA90EF324D96E32
:100FF800000EF420DA6EDECF13F0DDCF14F0040E0D
:101008001318156E1450166E1750020DA90EF324FE
:10101800D96E000EF420DA6E15C0DEFF16C0DDFFB3
:1010280018C00FF019C010F0120019501A101B1038
:101038001C10D8A402D0010E01D0000E1F6E0001B2
:10104800C505D8A405D01F04D8A402D0000E1200EC
:101058001950000168191FE11A50000169191BE1B4
:101068001B5000016A1917E11C5000016B19D8A424
:1010780012D00001C905D8A407D02A0E0001C4194E
:10108800D8B409D0000E12002A0E0001C419D8A441
:1010980002D0000E120000016851195C000169516C
:1010A8001A5800016A511B5800016B511C58D8B0DE
:1010B80002D0010E01D0000E1D6E020E0001C919EA
:1010C800D8A419D02A0E0001C419D8B405D01F50CD
:1010D800D8A402D0050E08D00001C505D8B414D094
:1010E8001F04D8A403D005D01E6E1AD01D04D8A49E
:1010F800F1D7040EF9D72A0E0001C419D8B40ED0BE
:101108000001C505D8A402D0010EEED71F04D8B43B
:1011180003D01D04D8A402D0020EE6D7030EE4D7EC
:101128001E5054EC04F01E50120004012039E8321D
:10113800030B0009D8A4120044D0548E080E0001F5
:10114800D06F1200BEEC03F0120089EC7FF01200A1
:10115800DE0E516E000E526E5480010E556E548E86
:101168001200AEEC0AF0120039EC7EF01200040115
:101178002451010DDF0EF324516E000EF420526E3F
:101188005480010E556E548E1200548E0401245161
:10119800010DDF0EF324D96E000EF420DA6E22C49E
:1011A800DFFF1200000E1F6E020E1E6E000E206E74
:1011B800000E216E000E236E000E226EDBEC0CF08A
:1011C800120004012151000AD8B4CBD7010AD8B4BF
:1011D800CBD7020AD8B4C8D7060AD8B4AED7030A00
:1011E800D8B4B0D7010AD8B4DDD70F0AD8B4B0D76D
:1011F800010AD8B4AAD7030AD8B4B9D7010AD8B40F
:10120800C4D7070A1200040120511F0BE806D8A40E
:10121800120004012451D8A4120058D0040122510C
:1012280004012311D8A41200040126510401271136
:10123800D8A41200000E0001C96F0001C469000E95
:101248000001C66F000E0001C86F010E0001C36FD8
:10125800ABC01AF0ACC01BF01A501B10D8B40AD09F
:10126800ABC01CF0ACC01DF01CC0D9FF1DC0DAFF1C
:10127800DFBE0FD0000E0F6E300E106E040E116E12
:10128800400E126E010E98EC07F00FC0B6F010C0B9
:10129800B7F0800E546E120004012251040123118C
:1012A800D8A412000401260504012711D8A41200AD
:1012B800000E0401286F280E516E040E526E000EA7
:1012C800566E010E556EC10E546E12000401215166
:1012D800FE0AD8B4E1D7010AD8A412009FD7080E95
:1012E8000F6E565013E1080E555CD8B00FD055C09C
:1012F8000FF00001D851D8A402D0010E05D000018A
:10130800D805D8A403D0020E0001D86F0F50555E3F
:10131800000E565A20EE01F05750D9265850DA22BE
:101328000FC0DFFF280E0001BE6F040E0001BF6F63
:1013380054A01CD03AD051C0F6FF52C0F7FFF86A4B
:10134800BEC0D9FFBFC0DAFF0E0EF76403D0080095
:10135800F55005D0F6CFE1FFF7CFE2FFE750DF6E9B
:10136800514A522A0001BE4BBF2B0F060F50D8B46A
:101378001200E1D751C0F6FF52C0F7FFF86ABEC0AD
:10138800D9FFBFC0DAFF0E0EF76403D00800F5508E
:1013980005D0F6CFE1FFF7CFE2FFE750DF6E514A05
:1013A800522A0001BE4BBF2B0F060F50D8B41200B3
:1013B800E1D70001D151D8A41200010E0001D16F6C
:1013C8000001D251D8A41200010E0001D26F020E02
:1013D8000001D519D8A415D020EE01F05750D92610
:1013E8005850DA22000EDF6E57C0D9FF58C0DAFF16
:1013F800480EDF6E57C0D9FF58C0DAFF000EDB8EEB
:1014080012000001D505D8A41200000E0001C26F19
:1014180020EE01F05B50D9265C50DA22080EDF6E10
:1014280020EE02F05B50D9265C50DA22200EDE6EE8
:10143800040EDD6E5BC0D9FF5CC0DAFF040EDF6E00
:101448005BC0D9FF5CC0DAFF000EDB8E010E000125
:10145800C26F20EE01F05D50D9265E50DA22080EE8
:10146800DF6E20EE02F05D50D9265E50DA22200EA3
:10147800DE6E040EDD6E5DC0D9FF5EC0DAFF800E41
:10148800DF6E120057C0D9FF58C0DAFF000EDFBC6C
:10149800010E106E040E5718576E5850586E080EED
:1014A8000001D019D8A40ED0040122517F0B0F01DE
:1014B800386F0F013851D8B402D0100E01D0040E85
:1014C8000001D06F0001D505D8A43BD020EE02F072
:1014D8005750D9265850DA22280EDE6E040EDD6EDB
:1014E80073EC09F0020E0001D819D8A40DD057C02A
:1014F800D9FF58C0DAFF040EDF6E57C0D9FF58C0B5
:10150800DAFF000EDB8E12001050D8A40DD057C0A1
:10151800D9FF58C0DAFF480EDF6E57C0D9FF58C050
:10152800DAFF000EDB8E120057C0D9FF58C0DAFF71
:10153800080EDF6E57C0D9FF58C0DAFF000EDB8EE9
:101548001200000194AF02D00001949F000E000128
:10155800D56F1200000E0401286F000E0401296FD8
:101568003BD0548E040128810001CA05D8A440D07C
:10157800040128833DD0548E3BD0548E040124BFEF
:101588000BD0040124510F0B0F6E0F50020DA90E42
:10159800F324D96E000E0AD0040124510F0B0F6EEC
:1015A8000F50020D570EF324D96E000EF420DA6E98
:1015B800DECF10F0DDCF11F010C0D9FF11C0DAFF77
:1015C800DFAE16D010C0D9FF11C0DAFFDFA410D0EB
:1015D800010E0401286F0CD0040120511F0B000AD2
:1015E800D8B4BFD7010AD8B4C6D7030AD8B4C5D768
:1015F80054AE1200280E516E040E526E5480020E24
:10160800556E12002D0E0001D36FE0C02CF0FD0EB8
:101618002C16D8A444D0E0C02CF0D8902C323F0E21
:101628002C162C50040D000EF3245B6E040EF420CF
:101638005C6E5BC05DF05CC05EF0040E5D185D6EB4
:101648005E505E6E5BC0D9FF5CC0DAFFDF30E83207
:101658000F0B0D0AD8A420D0200E0F6E040E106EAA
:1016680020EE02F05B50D9265C50DA22DECF2CF057
:10167800DDCF2DF02CC011F02DC012F0115012103A
:10168800D8A4200E136E000E156E080E146E75EC9D
:101698000DF0B0EC0BF0120043EC0DF0120000015D
:1016A800E051FD0B040AD8A4120046EC0AF012001F
:1016B8000F50116E1050126E136A146A1150000107
:1016C800685D125000016959135000016A5914509D
:1016D80000016B59D8B00ED0000E0401786F000ECF
:1016E800796F000E7A6F000E7B6F68C0B2F069C028
:1016F800B3F012000001B2510F5C0001B351105851
:10170800D8B004D00FC0B2F010C0B3F00001B2518D
:10171800116E0001B351126E136A146A111E121E63
:10172800131E141E112A000E122213221422000165
:10173800685111240401786F0001695112200401D5
:10174800796F00016A51132004017A6F00016B510F
:10175800142004017B6F1200000E0001D86F000EE8
:101768000001CF6F000E0001CD6F000E0001CE6F9B
:10177800000E0001C26F000E0001D56F57C0D9FFDF
:1017880058C0DAFF7F0EDF16040E5718576E5850F0
:10179800586E57C0D9FF58C0DAFF7F0EDF16040E07
:1017A8005718576E5850586E5DC0D9FF5EC0DAFFA3
:1017B8007F0EDF16000E546E000E566E000E556E2C
:1017C800000E0001946F000E0001966F000E956FD9
:1017D80099EC08F0000E1F6E030E1E6E000E206EB0
:1017E800000E216E000E236E000E226EDBEC0CF054
:1017F8008FEC06F01200000E0001CD6F000E000104
:10180800CE6F020E0001D519D8A41FD020EE01F02A
:101818005D50D9265E50DA22080EDF6E20EE02F007
:101828005D50D9265E50DA22280EDE6E040EDD6E7B
:101838005DC0D9FF5EC0DAFF480EDF6E5DC0D9FF1C
:101848005EC0DAFF000EDB8E120055500401265DE3
:10185800565004012759D8B004D026C455F027C4DF
:1018680056F073EC09F020EE02F05750D926585084
:10187800DA22280EDE6E040EDD6E57C0D9FF58C07E
:10188800DAFF480EDF6E57C0D9FF58C0DAFF000EE6
:10189800DB8E1200146E000E156E040E166E0F50BD
:1018A800106E116AD890103611361450126E136AE1
:1018B800D89012361336D890123613361050122696
:1018C80011501322D89012361336D8901236133688
:1018D800125015261350162215C0D9FF16C0DAFF6C
:1018E800DF9E0F50D8A407D01450020DA90EF32480
:1018F800D96E000E06D01450020D570EF324D96E7F
:10190800000EF420DA6E15C0DEFF16C0DDFF15C02C
:10191800D9FF16C0DAFFDF9C20EE04F01550D92657
:101928001650DA22DF8C120000017F917F937F9599
:101938007F977F897F8B7F8D00017F9F000E00013D
:10194800806F000181918193819581970001819B2E
:101958000001819D0001819F000E0001826F000E31
:101968000001836F000E0001846F000E0001856F77
:101978000A0E0001866F000E0001876F000E886F47
:10198800000E896F000E8A6F000E00018B6F000E2B
:1019980000018C6F000E00018D6F000E00018E6F2C
:1019A800000E00018F6F000E0001906F12000DD025
:1019B80041EC0FF0120007EC09F0120020C01AF0F9
:1019C80021C01BF000EC0EF012001EC024F01FC056
:1019D80025F02550000AD8B404D07F0AD8A41200F4
:1019E80018D02450010AD8B4E3D7030AD8B4120097
:1019F800010AD8B4E0D7060AD8B4E0D7770AD8B431
:101A08001200010AD8B41200070AD8B41200010A59
:101A180012002450FF0A120020D098EC0CF00001AC
:101A28008151F00B0209816F3A0E00018B6F000E95
:101A380000018C6F77EC79F01200010E04017C6FC5
:101A48000001C469120077EC79F0120077EC79F0A4
:101A580012007F0E54EC04F012000001C451000A79
:101A6800D8B4EBD7030AD8B4D8D7110AD8B4EBD76F
:101A78000C0AD8B4E2D7E30AD8B4E8D7EAD7020EFA
:101A88000001D519D8A403D002EC06F01200000E0C
:101A98000001D56F0001C251D8A41FD020EE01F07B
:101AA8005D50D9265E50DA22080EDF6E20EE02F075
:101AB8005D50D9265E50DA22200EDE6E040EDD6EF1
:101AC8005DC0D9FF5EC0DAFF0C0EDF6E5DC0D9FFC6
:101AD8005EC0DAFF000EDB8E1200000E0001C26F3E
:101AE800120011C016F012C017F013C018F00FC082
:101AF80019F010C01AF01DD016C0F6FF17C0F7FF76
:101B080018C0F8FF19C0D9FF1AC0DAFFF8BA03D015
:101B18000800F55005D0F6CFE1FFF7CFE2FFE75018
:101B2800DF6E010E1626000E1722000E1822194A23
:101B38001A2A1406D8A015061428DEE11528D8B4E8
:101B48001200DAD720501F101E1004E1690E1D5C28
:101B5800D8A002D0000E120021C00FF022C010F051
:101B68001DC023F01EC024F0090ED8902336243659
:101B7800E82EFBD7000E256E200E266E000E276E6F
:101B880023502524116E24502620126E000E272083
:101B9800136E020E156E000E146E75EC0DF0010E2C
:101BA800120008EE00F014EE00F0EE6AE550E15085
:101BB800FCE1E250FAE100EE60F0810EEE6AE80620
:101BC800FDE100EE51F00E0EEE6AE806FDE1480E6A
:101BD800F66E1E0EF76E000EF86E00EEE1F010EED7
:101BE80014F00900F5CFEEFFE550E150FAE15F90FF
:101BF8005F920001F9EF0EF00001C351D8A40BD099
:101C0800010E0F6E010E15EC07F0000E0F6E010E9F
:101C180015EC07F01200ABC01CF0ACC01DF01C5056
:101C28001A1814E11D501B18D8A41200000E0F6ECC
:101C3800300E106E040E116E400E126E010E98ECEE
:101C480007F00FC0B6F010C0B7F0120012000F0175
:101C580026A11ED05BC0D9FF5CC0DAFF800EDE185B
:101C6800D8A414D057C0D9FF58C0DAFF840EDE18A4
:101C7800D8A40CD05BC0D9FF5CC0DAFF0C0EDF6EB5
:101C88005BC0D9FF5CC0DAFF000EDB8E0F01269126
:101C9800629A12001A6E17A405D0000E0F6E1A5021
:101CA8004EEC0CF017A205D0010E0F6E1A504EEC38
:101CB8000CF01A50010D260EF324186E0F0EF420A6
:101CC800196E18C0D9FF19C0DAFF17C0DFFF12005C
:101CD800000E0001CC6F000E1F6E740E1E6E000EFB
:101CE800206E000E216E000E236E000E226EDBECBD
:101CF8000CF065920F01369501D0629462B4FDD75D
:101D0800000E0001D46F12000F01368562986582BB
:101D1800010E0001CC6F000E0001D46F000E1F6E83
:101D2800750E1E6E000E206E000E216E000E236EC4
:101D3800000E226EDBEC0CF012000F6E4EEC0FF072
:101D48000009D8B41200B50E0F18D8B402D0A69462
:101D58001200F2CF10F0F29E550EA76EAA0EA76ED3
:101D6800A682A69410AE1200F28E12000FC015F0D3
:101D780010C016F008D015C0D9FF16C0DAFF11C080
:101D8800DFFF154A162A1306D8A014061328F3E114
:101D98001428D8B41200EFD79B8C020E196E580E77
:101DA800186E1806D8A019061828FBE11928D8A417
:101DB800F8D70F0148693F0E0F01496F0EEC03F089
:101DC8001200010E00019D27000E9E239F23A023D1
:101DD8000001CC51D8A412000001D42B0001D45129
:101DE800D8A412000001D4691200D0EC0EF00EEC59
:101DF80003F041EC02F0200E0001D06101D0F9D7C8
:101E080065B2F7D72EEC0FF0F4D70001DA81020E95
:101E18000001DC6F000EDB6F000E0001D96FD90ED8
:101E28000F6E000E106E120011C0F6FF12C0F7FF01
:101E380013C0F8FF940EA66EB50EA1EC0EF01200BA
:101E4800121E701E921EA01E4C1BF4FF8200000082
:101E580000000000200E0001D06101D0120065B220
:101E68001200E8EC7CF01200680E0F6E000E106E87
:101E7800000E116E000E126E12001E0E176E010E6D
:101E88004EEC0EF075EC05F01200020E106E000E0E
:0C1E98000F6E1200010E1200010E12006D
:1020000000000000000000000000000000000000D0
:1020100000000000000000000000000000000000C0
:1020200000000000000000000000000000000000B0
:1020300000000000000000000000000000000000A0
:102040000000000000000000000000000000000090
:102050000000000000000000000000000000000080
:102060000000000000000000000000000000000070
:102070000000000000000000000000000000000060
:102080000000000000000000000000000000000050
:102090000000000000000000000000000000000040
:1020A0000000000000000000000000000000000030
:1020B0000000000000000000000000000000000020
:1020C0000000000000000000000000000000000010
:1020D0000000000000000000000000000000000000
:1020E00000000000000000000000000000000000F0
:1020F00000000000000000000000000000000000E0
:1021000000000000000000000000000000000000CF
:1021100000000000000000000000000000000000BF
:1021200000000000000000000000000000000000AF
:10213000000000000000000000000000000000009F
:10214000000000000000000000000000000000008F
:10215000000000000000000000000000000000007F
:10216000000000000000000000000000000000006F
:10217000000000000000000000000000000000005F
:10218000000000000000000000000000000000004F
:10219000000000000000000000000000000000003F
:1021A000000000000000000000000000000000002F
:1021B0000000000000000000F58B16EA000080011E
:1021C00001000107FFE601000000680000000000B8
:1021D00000000000000000000000000000000000FF
:1021E00000000000000000000000000000000000EF
:1021F000000000000000000000000000000055AAE0
:10220000EB3C904D53444F53352E300002010100FA
:102210000110000000F801003F00FF000100000075
:1022200068000000000029326794C44E4F204E41E0
:102230004D452020202046415431322020200000EE
:10224000000000000000000000000000000000008E
:10225000000000000000000000000000000000007E
:10226000000000000000000000000000000000006E
:10227000000000000000000000000000000000005E
:10228000000000000000000000000000000000004E
:10229000000000000000000000000000000000003E
:1022A000000000000000000000000000000000002E
:1022B000000000000000000000000000000000001E
:1022C000000000000000000000000000000000000E
:1022D00000000000000000000000000000000000FE
:1022E00000000000000000000000000000000000EE
:1022F00000000000000000000000000000000000DE
:1023000000000000000000000000000000000000CD
:1023100000000000000000000000000000000000BD
:1023200000000000000000000000000000000000AD
:10233000000000000000000000000000000000009D
:10234000000000000000000000000000000000008D
:10235000000000000000000000000000000000007D
:10236000000000000000000000000000000000006D
:10237000000000000000000000000000000000005D
:10238000000000000000000000000000000000004D
:10239000000000000000000000000000000000003D
:1023A000000000000000000000000000000000002D
:1023B000000000000000000000000000000000001D
:1023C000000000000000000000000000000000000D
:1023D00000000000000000000000000000000000FD
:1023E00000000000000000000000000000000000ED
:1023F000000000000000000000000000000055AADE
:10240000F8FFFFFF0F0000000000000000000000C8
:1024100000000000000000000000000000000000BC
:1024200000000000000000000000000000000000AC
:10243000000000000000000000000000000000009C
:10244000000000000000000000000000000000008C
:10245000000000000000000000000000000000007C
:10246000000000000000000000000000000000006C
:10247000000000000000000000000000000000005C
:10248000000000000000000000000000000000004C
:10249000000000000000000000000000000000003C
:1024A000000000000000000000000000000000002C
:1024B000000000000000000000000000000000001C
:1024C000000000000000000000000000000000000C
:1024D00000000000000000000000000000000000FC
:1024E00000000000000000000000000000000000EC
:1024F00000000000000000000000000000000000DC
:1025000000000000000000000000000000000000CB
:1025100000000000000000000000000000000000BB
:1025200000000000000000000000000000000000AB
:10253000000000000000000000000000000000009B
:10254000000000000000000000000000000000008B
:10255000000000000000000000000000000000007B
:10256000000000000000000000000000000000006B
:10257000000000000000000000000000000000005B
:10258000000000000000000000000000000000004B
:10259000000000000000000000000000000000003B
:1025A000000000000000000000000000000000002B
:1025B000000000000000000000000000000000001B
:1025C000000000000000000000000000000000000B
:1025D00000000000000000000000000000000000FB
:1025E00000000000000000000000000000000000EB
:1025F00000000000000000000000000000000000DB
:102600004472697665204E616D6520080000000007
:102610000011001100000000001100000000000087
:1026200046494C4520202020545854200006287844
:10263000DE38DE3800000477DE38020004000000D7
:10264000000000000000000000000000000000008A
:10265000000000000000000000000000000000007A
:10266000000000000000000000000000000000006A
:10267000000000000000000000000000000000005A
:10268000000000000000000000000000000000004A
:10269000000000000000000000000000000000003A
:1026A000000000000000000000000000000000002A
:1026B000000000000000000000000000000000001A
:1026C000000000000000000000000000000000000A
:1026D00000000000000000000000000000000000FA
:1026E00000000000000000000000000000000000EA
:1026F00000000000000000000000000000000000DA
:1027000000000000000000000000000000000000C9
:1027100000000000000000000000000000000000B9
:1027200000000000000000000000000000000000A9
:102730000000000000000000000000000000000099
:102740000000000000000000000000000000000089
:102750000000000000000000000000000000000079
:102760000000000000000000000000000000000069
:102770000000000000000000000000000000000059
:102780000000000000000000000000000000000049
:102790000000000000000000000000000000000039
:1027A0000000000000000000000000000000000029
:1027B0000000000000000000000000000000000019
:1027C0000000000000000000000000000000000009
:1027D00000000000000000000000000000000000F9
:1027E00000000000000000000000000000000000E9
:1027F00000000000000000000000000000000000D9
:10280000446174610000000000000000000000004E
:1028100000000000000000000000000000000000B8
:1028200000000000000000000000000000000000A8
:102830000000000000000000000000000000000098
:102840000000000000000000000000000000000088
:10F2000000E9F245F20BF2BDF29DF23A034D0069BE
:10F2100000630072006F00630068006900700020E6
:10F22000004D006100730073002000530074006FF4
:10F2300000720061006700650020004400720069F0
:10F24000007600650034034D006900630072006FB2
:10F2500000630068006900700020005400650063CE
:10F260000068006E006F006C006F0067007900207E
:10F270000049006E0063002E0000800402200000A0
:10F2800000426F626F724B65794D617373205374E6
:10F290006F726167652020202030303031090220F4
:10F2A00000010100C03209040000020806500007F6
:10F2B000058102400001070501024000011A0331E7
:10F2C0000032003300340035003600370038003992
:10F2D000003000390039001201000200000008D897
:10F2E0000409000100010203010403090400D1D153
:10F2F00044EC01F00009D8A412000001C469120016
:10F300006EEC7BF00009D8A412000001C469120061
:10F310000001C505D8A403D00001C469120072C061
:10F32000B3F073C0B2F0B2C019F0B3C01AF01B6AE8
:10F330001C6A19EC08F00009D8A41200000E106E27
:10F34000240E0F6E5CEC0BF0000E0F6E060E106EAE
:10F35000790E116EF20E126E11501210D8A4000E1A
:10F36000136E000E156E240E146E75EC0DF0FD0E6E
:10F370000001C46F1200EFC00FF0F0C010F001D810
:10F380000AD00500FA6E0001E351FD6EE451FE6EF5
:10F39000FF6AFA5012000FC047F010C048F011C0C9
:10F3A00049F012C04AF0EFC00FF0F0C010F001D8E1
:10F3B0000AD00500FA6E0001E551FD6EE651FE6EC1
:10F3C000FF6AFA5012000FC043F010C044F0456AC3
:10F3D000466A26EE00F04AC0DFFF26EE01F049C083
:10F3E000DFFF26EE02F048C0DFFF26EE03F047C045
:10F3F000DFFF26EE04F046C0DFFF26EE05F045C035
:10F40000DFFF26EE06F044C0DFFF26EE07F043C024
:10F41000DFFF000E0001B36F080EB26F000E106E1A
:10F42000080E0F6E5CEC0BF0FD0E0001C46F1200B5
:10F430000001C505D8A403D00001C4691200000E64
:10F440000001B36F120EB26F000E106E120E0F6E2F
:10F450005CEC0BF0000E4B6E110E4B6401D014D01F
:10F460004B50010D7F0EF324D96E000EF420DA6E9E
:10F470004B50010D000EF324E16E060EF420E26EF7
:10F48000DFCFE7FF4B2AE8D7FD0E0001C46F120063
:10F49000030EE8CF00F6000EE8CF01F6EFC00FF044
:10F4A000F0C010F001D80AD00500FA6E0001EB514F
:10F4B000FD6EEC51FE6EFF6AFA5012000009D8A4EE
:10F4C00004D0000E416E000E03D0000E416E800E7F
:10F4D000406E26EE02F040C0DFFF000EE8CF03F6DC
:10F4E000000E0001B36F040EB26F000E106E040E1A
:10F4F0000F6E5CEC0BF0FD0E0001C46F12000001FA
:10F500008151F00B0509816F200E00018B6F000EF9
:10F5100000018C6F010E04017C6F000E0401786FF6
:10F52000000E796F000E7A6F000E7B6F0001C469C8
:10F530001200000E196E000E1A6E000E1B6E000EE9
:10F540001C6E19EC08F00009D8A4120000018151CA
:10F550000F0B060AD8A407D004017C05D8A403D059
:10F560000001C469120098EC0CF0000E0401786FE1
:10F57000000E796F000E7A6F000E7B6F0001C46978
:10F580001200000E0401786F000E796F000E7A6F82
:10F59000000E7B6F0001C46912000001B45100012C
:10F5A000B511D8B407D0B4C0D9FFB5C0DAFF000197
:10F5B000DFBE120000016B5100016A1100016911E8
:10F5C00005E1400E0001685DD8A00AD0400E426EF1
:10F5D000400E0001685F000E695B6A5B6B5B0BD0DD
:10F5E00068C042F0000E0001686F000E696F000EE7
:10F5F0006A6F000E6B6F42503E6E3F6A3E500001D4
:10F60000B25D3F500001B359D8A006D0425000016E
:10F61000B25F000EB35B1DD0000E4B6E16D0000122
:10F62000B2510001B311D8B405D00001B207D8A07F
:10F63000B3070AD04B50010D000EF324D96E060E0D
:10F64000F420DA6E000EDF6E4B2A42504B5CD8A0DD
:10F65000E6D7010E0F6E000E106E060E116E42C040
:10F6600012F0010E98EC07F00FC0B4F010C0B5F026
:10F67000000168510001691100016A1100016B115C
:10F68000D8A412000001C46912007F0E54EC04F0EB
:10F6900012000001C451000AD8B44BD7030AD8B4F1
:10F6A000C7D6110AD8B434D6080AD8B4F1D6010A9C
:10F6B000D8B467D7050AD8B422D73B0AD8B45BD6EA
:10F6C0000D0AD8B415D6020AD8B41AD6050AD8B489
:10F6D00058D7D20AD8B461D7030AD7D764D171C03A
:10F6E0009CF072C09BF073C09AF074C099F076C021
:10F6F000B3F077C0B2F00001B251396E0001B351DE
:10F700003A6E3B6A3C6A090ED89039363A363B3637
:10F710003C36E82EF9D739C019F03AC01AF03BC090
:10F720001BF03CC01CF019EC08F00009D8A44DD126
:10F73000EFC00FF0F0C010F001D80AD00500FA6E4B
:10F740000001EB51FD6EEC51FE6EFF6AFA501200A3
:10F750000009D8B419D0010E04017C6F0001815159
:10F76000F00B0709816F270E00018B6F000E00015F
:10F770008C6F000E0F6E010E15EC07F0000E0001ED
:10F78000C86F0001C8511200010E0001C96F0001CD
:10F79000B2510001B311D8B402D1030E0001C86FF9
:10F7A000000E0001C06F060E0001C16F000E0401C3
:10F7B000786F020E796F000E7A6F000E7B6F040176
:10F7C00078510401791104017A1104017B11D8B434
:10F7D00020D00001B6510001B711D8B407D0B6C08F
:10F7E000D9FFB7C0DAFF0001DFBEEFD0000E0F6E09
:10F7F000C0C010F0C1C011F0400E126E010E98ECA6
:10F8000007F00FC0B6F010C0B7F0040E0001C86FCB
:10F8100023D0EFC00FF0F0C010F001D80AD00500DF
:10F82000FA6E0001EB51FD6EEC51FE6EFF6AFA506C
:10F8300012000009D8B40ED0010E04017C6F000143
:10F840008151F00B0209816F270E00018B6F000EB2
:10F8500000018C6F020EA4D00001B6510001B71157
:10F86000D8B407D0B6C0D9FFB7C0DAFF0001DFBEF9
:10F87000ACD0000120EE01F0B651D926B751DA2202
:10F88000DF50396E39C03AF03B6A3C6A3D6A3A5003
:10F890000001685F3B500001695B3C5000016A5BFE
:10F8A0003D5000016B5B000120EE01F0B651D926FE
:10F8B000B751DA22DF50396E39C03AF03B6A3C6A00
:10F8C0003D6A3A500401785F3B500401795B3C503B
:10F8D00004017A5B3D5004017B5B400E0001C027B0
:10F8E000000EC123030E5CD004017C51D8A442D089
:10F8F000EFC01BF0F0C01CF099C01DF09AC01EF0C4
:10F900009BC01FF09CC020F0000E216E060E226EE0
:10F910000001995100019A1100019B1100019C11F5
:10F92000D8A402D0010E01D0000E236E01D80AD057
:10F930000500FA6E0001ED51FD6EEE51FE6EFF6A9C
:10F94000FA501200E806D8B415D0640E0001C76161
:10F9500003D00001C72B39D0010E04017C6F0001D8
:10F960008151F00B0309816F000E00018B6F000EB7
:10F9700000018C6F010E00019927000E9A239B2332
:10F980009C230001B207D8A0B307010E09D0020ED4
:10F9900004017C6F000E0F6E010E15EC07F0000ED7
:10F9A0000001C86F12D00001C851000AD8B497D620
:10F9B000010AD8B4ECD6030AD8B496D7010AD8B451
:10F9C000FED6070AD8B448D7E2D70001C8511200C2
:10F9D000200E0001D019D8A412003CD10001B6516C
:10F9E0000001B711D8B407D0B6C0D9FFB7C0DAFF4D
:10F9F0000001DFBE1200000E0001FA6F1E0E0001B2
:10FA0000FA6501D017D00001FA51010D300EF32430
:10FA1000D96E040EF420DA6E0001FA51010D600E69
:10FA2000F324E16E000EF420E26EDFCFE7FF000169
:10FA3000FA2BE4D7000120EE01F0B651D926B751D8
:10FA4000DA221F0EDE18D8A484D0550E00016019EA
:10FA50000CE1530E000161197CE1420E00016219B4
:10FA600078E1430E00016319D8A473D0010E0001A0
:10FA7000C36F00016D51D8A461D0110E00016E61F9
:10FA80005DD000016E51D8B459D06CC0F5F03F0E76
:10FA90000001F517D8A452D0550E0401706F530E13
:10FAA000716F420E726F530E736F64C074F465C051
:10FAB00075F466C076F467C077F4000E0401786FC1
:10FAC000000E796F000E7A6F000E7B6F000E04013E
:10FAD0007C6F0001C469000E0001C66F000E0001BA
:10FAE000C86F000E0001C76F030E00016F19D8B474
:10FAF0000BD000018191819381958197000E0001C7
:10FB00008B6F000E00018C6F00016CAF02D0010EF4
:10FB100001D0020E0001C96F000168510001691196
:10FB200000016A1100016B11D8B402D0000E01D09F
:10FB3000010E0001C56F6FC0C4F01200010E0F6E00
:10FB4000010E15EC07F0000E0F6E010E15EC07F01C
:10FB50001200010E0F6E010E15EC07F0000E0F6E75
:10FB6000010E15EC07F0000E0001C36F1200E5EC6A
:10FB700004F0FF0AD8A41200030E0001C96F12009E
:10FB8000E5EC04F0FF0AD8A4120004017C51D8A4CB
:10FB90000DD0040178510401791104017A11040196
:10FBA0007B11D8B403D0020E04017C6F030E000158
:10FBB000C96F120059C0F6F05AC0F7F00001F651B3
:10FBC0000001F711D8B40BD059C0F8F05AC0F9F0C1
:10FBD000F8C0D9FFF9C0DAFF0001DFBE1200010E44
:10FBE0000F6E700E106E040E116E0D0E126E010E61
:10FBF00098EC07F00FC0B4F010C0B5F00001B6519A
:10FC00000001B711D8B407D0B6C0D9FFB7C0DAFF2A
:10FC10000001DFBE0FD0000E0F6E300E106E040E0E
:10FC2000116E400E126E010E98EC07F00FC0B6F088
:10FC300010C0B7F0000E0001C96F1200000E0001E5
:10FC4000C96F020E04017C6F000E0F6E010E15ECE1
:10FC500007F012000001C951000AD8B4BFD6010A4A
:10FC6000D8B485D7030AD8B48BD7010AD8B4A2D7A1
:10FC7000E5D704012205D8A411D0040120511F0B9F
:10FC80000009D8A40BD0548E030E04012119D8A466
:10FC900002D0010E01D0000E0001CA6F04012251F2
:10FCA000D8A41200040120511F0B020AD8A412008C
:10FCB000040124510F0B0009D8B41200040124518F
:10FCC0000F0B266E020E26601200200E0001D019C6
:10FCD000D8A41200548E040124BF1BD00401245167
:10FCE0000F0B266E2650020DA90EF324D96E000EBE
:10FCF000F420DA6EDECF2AF0DDCF2BF004012451A0
:10FD00000F0B266E2650010DBA0EF324D96E000E8D
:10FD10001AD0040124510F0B266E2650020D570EE7
:10FD2000F324D96E000EF420DA6EDECF2AF0DDCF98
:10FD30002BF0040124510F0B266E2650010DB80E36
:10FD4000F324D96E000EF420DA6EDF50296E29B04C
:10FD500006D0FB0E2A142A6EFF0E2B1404D0040EBC
:10FD60002A102A6E2B502B6E040124BF0BD00401E5
:10FD700024510F0B266E2650020DA90EF324D96EC6
:10FD8000000E0AD0040124510F0B266E2650020DDE
:10FD9000570EF324D96E000EF420DA6E2AC0DEFF6F
:10FDA0002BC0DDFF030E04012119D8A42FD02AC0D7
:10FDB000D9FF2BC0DAFFDFAE1CD0040124BF0BD06B
:10FDC000040124510F0B266E2650010DBA0EF324A8
:10FDD000D96E000E0AD0040124510F0B266E265056
:10FDE000010DB80EF324D96E000EF420DA6E000176
:10FDF000DF822AC0D9FF2BC0DAFF000EDB842AC0C5
:10FE0000D9FF2BC0DAFF000EDB8E1200040E2A1879
:10FE10002A6E2B502B6E2AC0D9FF2BC0DAFFDFAE23
:10FE20001BD02AC0D9FF2BC0DAFF7F0EDF162AC0F5
:10FE3000D9FF2BC0DAFF000EDB8C000E1F6E050E03
:10FE40001E6E2AC020F02BC021F0000E236E020E81
:10FE5000226EDBEC0CF006D02AC0D9FF2BC0DAFFF3
:10FE6000000EDB8C040E2A182A6E2B502B6E29B242
:10FE700006D02AC0D9FF2BC0DAFFDFAE31D0040193
:10FE800024BF0BD0040124510F0B266E2650010D08
:10FE9000BA0EF324D96E000E0AD0040124510F0BC0
:10FEA000266E2650010DB80EF324D96E000EF420F4
:10FEB000DA6E0001DF922AC0D9FF2BC0DAFF3B0EB9
:10FEC000DF16000E1F6E050E1E6E2AC020F02BC01E
:10FED00021F0000E236E020E226EDBEC0CF006D039
:10FEE0002AC0D9FF2BC0DAFF3B0EDF1604012451D4
:10FEF0000F0B266E2650010D260EF324276E0F0ED3
:10FF0000F420286E27C0D9FF28C0DAFFFE0EDF16C6
:10FF10001200548E270E0F6E0F0E106E000E126E12
:10FF2000000E116E000E146E010E136EBAEC0EF080
:10FF3000000E0F6E040E106E000E126E000E116E8B
:10FF4000000E146E200E136EBAEC0EF0658C000ECF
:10FF5000266E010E266401D016D02650010DB80E73
:10FF6000F324D96E000EF420DA6E000EDF6E2650F8
:10FF7000010DBA0EF324D96E000EF420DA6E000ED5
:10FF8000DF6E262AE6D7DF0E0F6E000E106E000E13
:10FF9000126E000E116E000E146E010E136EBAEC8E
:10FFA0000EF0659C080E576E040E586E000E5B6EC8
:10FFB000040E5C6E5BC05DF05CC05EF022C4DEF0DF
:10FFC0000001DE51D8A404D0100E0001D06F120041
:10FFD000000E1F6E010E1E6EDE0E206E000E216ED4
:10FFE000000E236E010E226EDBEC0CF0200E0001E1
:08FFF000D06F1200000E120098
:08FFF800ACF71AFF63F881F178
:00000001FF
